:10165E0043B38053B47F43AC0153ADFE75F60343E1
:05166E00E101D2AE22F3
:10159F008C0B8D0C8B088A09890AE92402F9E43A2D
:1015AF00FAC003A80AAC09AD03D0037E007F0C126A
:1015BF00055EAB08AA09A90A90000CE50B850CF093
:0315CF000202769F
:1015D2000204060A10142028324050647EA0C8FE7D
:1015E2000780084008B1093F09C10A000A820AC0FF
:1015F2000AFE0B430B810BBF0BFF0C410C800CC28C
:10000E001210ADE4F51A751B14F51CF51D751F0ABB
:0F001E0043B30153B4FE53B3FD43B402D2912256
:100FF9009015D2E493FEEFC39E50059015E2800E42
:101009009015E1E493FEEFC39E400B901600E49324
:10101900FE740193FF22E4F50DE50DC3940F74806E
:1010290094805019E50D9015D293FEEFC39E4009A7
:10103900E50DA393FEEF9E4004050D80DCE50D90C0
:1010490015D293F9FDC3EF9DFFE49400FEE50D254C
:10105900E024E2F582E43415F583E493FC7401930A
:10106900FDE50D25E024E4F582E43415F583C37428
:1010790001939DFDE4939CFC1201ACE9FDE50D9003
:1010890015D393C39DFDE49400FC1201BEE50D2523
:10109900E024E2F582E43415F5837401932FFFE42B
:0310A900933EFE75
:0110AC002221
:100F1400D39015E27401939FEE6480F8E4936480A7
:100F24009840059015D28016D39016007401939FB3
:100F3400EE6480F8E49364809850079015E1E4939C
:100F4400FF22E4F508C3E508940F74809480503EB2
:100F5400E50825E024E2F582E43415F583D3740131
:100F6400939FEE6480F8E493648098501DE508250F
:100F7400E024E4F582E43415F583D37401939FEE01
:100F84006480F8E4936480985004050880B7E50809
:100F94009015D293FDE508A393C39DFDE49400FC52
:100FA400E50825E024E2F582E43415F583E493FAB8
:100FB400740193FBC3EF9BFFEE9AFE1201ACE508AC
:100FC40025E024E2F582E43415F583E493FC74010E
:100FD40093FDE50825E024E4F582E43415F583C3A4
:100FE4007401939DFDE4939CFC1201BEE5089015E9
:040FF400D2932FFF66
:010FF80022D6
:100BEB00D3900083E09F900082E09E4002800DD363
:100BFB00900089E09F900088E09E5005E4F5088006
:100C0B0044E4F508C3E5089401748094805036E5FC
:100C1B000875F006A42482F582E43400F583E0FC29
:100C2B00A3E0D39FEC9E5019E50875F006A4248829
:100C3B00F582E43400F583E0FCA3E0D39FEC9E50F7
:100C4B0004050880BFE4FCFDC006C007E50875F08D
:100C5B0006A42482F582E43400F583E0FEA3E0FBD6
:100C6B00AA06D007D006C3EF9BFBEE9AFAED9400D1
:100C7B00F9EC9400F8E50875F006A42480F582E4FD
:100C8B003400F583E0FEA3E0FFE50875F006A4242D
:100C9B0086F582E43400F583E0FCA3E0C39FFFEC10
:100CAB009EFE3395E0FDFC1202A3C004C006C007F4
:100CBB00E50875F006A42482F582E43400F583E0A0
:100CCB00FEA3E0FFE50875F006A42488F582E43462
:100CDB0000F583E0FCA3E0C39FFFEC9EAB07FAE4B7
:100CEB00F9F8D007D006D0041214A0E50875F00669
:100CFB00A42480F582E43400F583E0FCA3E02FFF0D
:030D0B00EC3EFEBD
:010D0E0022C2
:10113000E51DC3135403FBE4F519751A01AF19C378
:10114000EF940F7480948040F4E51D30E50CAF1EE1
:10115000EF75F040A4FFAEF08008E51E25E0FF1219
:101160000FF9EB75F006A42480F582E43400F583D2
:10117000EEF0A3EFF0EB75F006A42482F582E434E0
:1011800000F583E54FF0A3E550F0EB75F006A424DD
:1011900084F582E43400F583E53DF0A3E53EF0AF4D
:0F11A00003EB64017003121673531DF7E4F51A85
:0111AF00221D
:1010AD00D201750E01750F00751080E4F50DC3E5C5
:1010BD000D940C748094805035E4250DFFE434407C
:1010CD00FE1216ADAB0EAA0FA910EF12019A300148
:1010DD000EAB0EAA0FA910120154F46002C20174D6
:1010ED00012510F510E4350FF50F050D80C0300109
:1010FD00319000807407F0A37480F0A37408F0A3FE
:10110D007432F0A37405F0A304F0A3740CF0A3746F
:10111D0080F0A3740AF0A37496F0A37407F0A3747F
:02112D008DF043
:01112F00229D
:101673007B017A00798075120C7F007E40020E197F
:1015660053B1BF53B2BF53B17F53B27F7598504347
:101576008920438780438E1053C4DFAB07AA06A990
:1015860005A8047F407E427D0F7C0012032EEF04E7
:09159600F404F58DD28ED29922E5
:1011B0008F5C8E5B8D5A8C5953B1BF53B2BF53B104
:1011C0007F53B27F75985043878053C4F843C4203F
:1011D000AB5CAA5BA95AA8597F407E427D0F7C0078
:1011E00012032EC374FF9FFF74FF9EFEE49DFDE477
:1011F0009CFC78081203D18FC6AB5CAA5BA95AA8E5
:10120000597F407E427D0F7C0012032EC374FF9FE6
:09121000FF8FC543C408D29922E6
:070003003098FDAF99C2988F
:01000A0022D3
:08169500C2998F993099FD22E2
:101219008F608E5F8D5E8C5D53B1FB53B2FB53B310
:10122900BF53B4BF75F85075C40853C4DFAB60AA87
:101239005FA95EA85D7F407E427D0F7C0012032E70
:10124900C374FF9FFF74FF9EFEE49DFDE49CFC7840
:10125900081203D18FC6AB60AA5FA95EA85D7F4063
:101269007E427D0F7C0012032EC374FF9FFF8FC542
:0412790043C4082240
:07169D0030F8FDAF9AC2F81E
:0116A4002223
:0816A500C2F98F9A30F9FD2211
:1013BF008F648E638D628C61538EF7438901D28C5B
:1013CF00E4FFFEFDFCAB64AA63A962A861C312032C
:1013DF00C06025758A7E758CFF308DFDC28DE564EA
:1013EF0024FFF564E56334FFF563E56234FFF562CE
:0B13FF00E56134FFF56180C8C28C225C
:10140A008F688E678D668C65538EF7438901D28CFF
:10141A00E4FFFEFDFCAB68AA67A966A865C31203D0
:10142A00C06025758ACA758CFA308DFDC28DE56853
:10143A0024FFF568E56734FFF567E56634FFF5666E
:0B144A00E56534FFF56580C8C28C2208
:101455008F6C8E6B8D6A8C69538EEF438910D28E9B
:10146500E4FFFEFDFCAB6CAA6BA96AA869C3120375
:10147500C06025758BEA758DCB308FFDC28FE56C0D
:1014850024FFF56CE56B34FFF56BE56A34FFF56A0F
:0B149500E56934FFF56980C8C28E22B3
:101371008F708E6F8D6E8C6D53C9BF53C9DF43C99A
:1013810010D2CAE4FFFEFDFCAB70AA6FA96EA86D76
:10139100C31203C0602575CC3075CDF830CFFDC2C6
:1013A100CFE57024FFF570E56F34FFF56FE56E341E
:0E13B100FFF56EE56D34FFF56D80C8C2CA22EF
:1012D1008F748E738D728C7175C40743C408E4FFDB
:1012E100FEFDFCAB74AA73A972A871C31203C0609E
:1012F1002B75C52C75C6CFE5C45410641070F85316
:10130100C4EFE57424FFF574E57334FFF573E572FA
:1013110034FFF572E57134FFF57180C253C4F722D1
:101321008F788E778D768C7575C40743C408E4FF7A
:10133100FEFDFCAB78AA77A976A875C31203C0603D
:101341002B75C5D875C6FFE5C45410641070F853E9
:10135100C4EFE57824FFF578E57734FFF577E57696
:1013610034FFF576E57534FFF57580C253C4F72275
:10003600E4F55153B3F753B4F753B3EF53B4EFD2D8
:0E00460094D29375C128D2C6D2C2439B012228
:10127D00EF14B40D00504A90129275F003A4C5837B
:10128D0025F0C583730212B90212CB0212BC0212F1
:10129D00BF0212CB0212CB0212CB0212CB0212C230
:1012AD000212C50212C80212CB0212CB7F02227F9C
:1012BD0004227F03227F02227F02227F00227F01F0
:0412CD00227F00225A
:030033000208AB15
:1008AB00C0E0C0F0C083C082C0D075D000C000C013
:1008BB0001C002C003C004C005C006C007AFBDEF36
:1008CB0024A0603624E0604224E07003020A632413
:1008DB00F8700302099E24F07003020A3F24F8709B
:1008EB0003020A6324F87003020A6324C86003023C
:1008FB000A65755100D2C4020A65AF51EF6003025D
:10090B000A65755101D2C2020A65AF51EF640170DD
:10091B002885BC52755102AF5212127D8F53AF53C3
:10092B00EF700EE55224F57008D291531DEF7551FF
:10093B0000755400D2C2020A65AF51EF6402600A1F
:10094B00AF51EF64036003020A65AF5474552FF87F
:10095B00A6BC0554E554C395535005755103802E21
:10096B00E55224F9601124FE601224FD601A24075D
:10097B00701985551D801485551E800FAF56EFAD30
:10098B0055F51BEDF51C800385551F755100D2C223
:10099B00020A65AF51EF64026003020A65755104E8
:1009AB00E55224FE602214602414603924FE605842
:1009BB0024FE605924FE605A24FD605F240C705E97
:1009CB0075550375560180567555018051C2AEAFF2
:1009DB0050EFF555E54FF556AF3EEFF557E53DF5C5
:1009EB0058D2AE8039C2AE851855E5555401AD5578
:1009FB002DFFE433A2E713EF13F555AF7CEFF5565C
:100A0B00E57BF557D2AE8016851D558011851E5599
:100A1B00800CAF1CEFF555E51BF556851F55AF54F4
:100A2B0074552FF8E6F5BC0554E554C39553502186
:100A3B00D2C28026AF51EF6404701FAF5474552F90
:100A4B00F8E6F5BC0554E554C395535004D2C28067
:100A5B0009755100C2C28002D2C2C2C3D007D006F0
:100A6B00D005D004D003D002D001D000D0D0D0829A
:070A7B00D083D0F0D0E0327F
:03000B000214E4F8
:1014E400C0E0C0F0C083C082C0D075D000C000C0CE
:1014F40001C002C003C004C005C006C00753E8F021
:10150400D2EE12168CC28DD007D006D005D004D0EE
:1015140003D002D001D000D0D0D082D083D0F0D07C
:02152400E032B3
:03005B00020A8214
:100A8200C0E0C0F0C083C082C0D075D000C000C03A
:100A920001C002C003C004C005C006C007E5E85497
:100AA2000F7027FB7A007941AFC3EF75F010A4FFF6
:100AB200ADC2E5F0FCEF4DFD12159FE5E854F044A0
:100AC20001F5E8D2EEC2EF020BD0E5E8540F640163
:100AD2006003020BCEFB7A007921AFC3EF75F010F1
:100AE200A4FFADC2E5F0FCEF4DFD12159F782F7CFF
:100AF200007D007B007A0079417E007F0E12012E7C
:100B02007B007A00792F1205DB8E4F8F50782F7C75
:100B1200007D007B007A0079217E007F0E12012E7B
:100B22007B007A00792F1205DB8E3D8F3ED3E55094
:100B3200953EE54F953D400CE550953EFFE54F95BE
:100B42003DFE80047E007F008E3F8F40AF40AE3F6F
:100B5200120D0F8E7B8F7CAF50AE4F120BEB8E16A9
:100B62008F17AF17AE16120F148F18AF1AEF64015A
:100B720070020519E51D20E04DE51D20E448309086
:100B820045E518D3951F403EAF797E00EF94097476
:100B92008094804011E57A9407748094804027C243
:100BA20091431D108020D3E57C951CE57B951B406D
:100BB20006057A05798015D3EF9400EE648094805F
:100BC200400A05798006757900757A00C2EFD00770
:100BD200D006D005D004D003D002D001D000D0D0AE
:090BE200D082D083D0F0D0E032C3
:1016020012165E12000E12003612168343B702C281
:10161200B953B7BFD2BE53F7FE53EFFED2AF121685
:101622008CAF1AEF70FBE51D30E3F612113080F13A
:101526000000003E005D007C009B00BA00D900F878
:1015360001360193020F026C030703A2043D0573F3
:10154600FFFF45CB2EC8235A1C8E181314EA12959A
:101556000F660C9D0AA109C708F40885084A080009
:100D0F00D39015447401939FE4939E500B901564F8
:100D1F00E493FE740193FF22E4F508C3E508940FF2
:100D2F00748094805032E50825E02426F582E4345F
:100D3F0015F583D37401939FE4939E5017E508250F
:100D4F00E02428F582E43415F583D37401939FE4EE
:100D5F00939E5004050880C3E4FCFDC006C007E560
:100D6F000825E02426F582E43415F583E493FE7418
:100D7F000193FBAA06D007D006C3EF9BFBEE9AFAAE
:100D8F00ED9400F9EC9400F8E50825E02448F5828D
:100D9F00E43415F583E493FE740193FFE50825E031
:100DAF002446F582E43415F583C37401939FFFE461
:100DBF00939EFEE41202A3C006C007E50825E024B7
:100DCF0026F582E43415F583E493FE740193FFE571
:100DDF000825E02428F582E43415F583C3740193C4
:100DEF009FFFE4939EAB07FAE4F9F8D007D0061201
:100DFF00032EE50825E02446F582E43415F583C378
:090E0F007401939FFFE4939EFE21
:010E180022B7
:091683004389015389FDD2A9221B
:09168C00758A95758CF5D28C224B
:1005DB0090000A12021FFFAEF01201F4FDACF0D333
:0505EB009FEC9E401D85
:1005F0008C088D0990000A12021FFFE5F08FF0129F
:0D060000025790000AE5088509F012027605
:10060D0090000612021FFFAEF01201F4FDACF0D304
:05061D009FEC9E401D52
:100622008C088D0990000612021FFFE5F08FF01270
:0D0632000257900006E5088509F0120276D7
:10063F0090000C12021FFFAEF090000212021FFD7D
:08064F00ACF0D39FEC9E4020AB
:100657008C088D0990000C12021FFF900002E5F034
:100667008FF012027690000CE5088509F0120276E9
:1006770090000812021FFFAEF090000412021FFD47
:08068700ACF0D39FEC9E402073
:10068F008C088D0990000812021FFF900004E5F0FE
:10069F008FF0120276900008E5088509F0120276B5
:1006AF0090000212021FFFAEF01201F4FDACF0D366
:0506BF009FEC9E401DB0
:1006C4008C088D0990000212021FFFE5F08FF012D2
:0D06D4000257900002E5088509F012027639
:1006E10090000A12021FFFAEF090000612021FFDD9
:0806F100ACF0D39FEC9E402009
:1006F9008C088D0990000A12021FFF900006E5F090
:100709008FF012027690000AE5088509F012027648
:1007190090000C12021FFFAEF090000412021FFDA0
:08072900ACF0D39FEC9E4020D0
:100731008C088D0990000C12021FFF900004E5F057
:100741008FF012027690000CE5088509F01202760E
:1007510090000612021FFFAEF090000412021FFD6E
:08076100ACF0D39FEC9E402098
:100769008C088D0990000612021FFF900004E5F025
:100779008FF0120276900006E5088509F0120276DC
:1007890090000C12021FFFAEF090000612021FFD2E
:08079900ACF0D39FEC9E402060
:1007A1008C088D0990000C12021FFF900006E5F0E5
:1007B1008FF012027690000CE5088509F01202769E
:1007C10090000A12021FFFAEF090000812021FFDF6
:0807D100ACF0D39FEC9E402028
:1007D9008C088D0990000A12021FFF900008E5F0AD
:1007E9008FF012027690000AE5088509F012027668
:1007F90090000812021FFFAEF090000212021FFDC6
:08080900ACF0D39FEC9E4020EF
:100811008C088D0990000812021FFF900002E5F07C
:100821008FF0120276900008E5088509F012027631
:1008310090000612021FFFAEF090000212021FFD8F
:08084100ACF0D39FEC9E4020B7
:100849008C088D0990000612021FFF900002E5F046
:100859008FF0120276900006E5088509F0120276FB
:1008690090000812021FFFAEF090000612021FFD51
:08087900ACF0D39FEC9E40207F
:100881008C088D0990000812021FFF900006E5F008
:100891008FF0120276900008E5088509F0120276C1
:0A08A10090000612021FFFAEF022C5
:0816AD008F828E83E493FF227B
:0A0E19008E0D8F0E8B0F8A108911C9
:100E2300E50E7807CEC313CE13D8F97807C333CEB4
:100E330033CED8F9F5158E14E4F513C3E513948076
:100E430074809480501F7E00E5152513FFEE351442
:100E5300FE1216AD74002513F582E43400F583EF1A
:100E6300F0051380D6E4F513E513C39512502CABAC
:100E73000FAA10A91185138275830012016DFFE576
:100E83000E547FFDE5132DFDE433FC74002DF58234
:100E930074003CF583EFF0051380CDC2AF75C7AA8C
:100EA30075C755439F0175C7AA75C75543A50175F6
:100EB300AF22E515F5A6E514F5A775AEFF75C7AA2C
:100EC30075C75543A40175AF21E4F513C3E5139426
:100ED30080748094805025E5152513F5A6E514F557
:100EE300A774002513F582E43400F583E0F5AE75AD
:100EF300C7AA75C75543A401051380D075C7AA7542
:100F0300C75553A5FE75C7AA75C755539FFED2AFE4
:010F130022BB
:03000000021632B3
:1016320075C7AA75C75575FD5A75C7AA75C7557579
:10164200FDA5787FE4F6D8FD9000007FFF7E03E4DD
:0C165200F0A3DFFCDEFA75817C021602BA
:10005E00E709F608DFFA8046E709F208DFFA803E84
:10006E0088828C83E709F0A3DFFA8032E309F60871
:10007E00DFFA8078E309F208DFFA807088828C83D9
:10008E00E309F0A3DFFA806489828A83E0A3F6088D
:10009E00DFFA805889828A83E0A3F208DFFA804C67
:1000AE0080D280FA80C680D4806980F2803380103E
:1000BE0080A680EA809A80A880DA80E280CA8033A7
:1000CE0089828A83ECFAE493A3C8C582C8CCC5831F
:1000DE00CCF0A3C8C582C8CCC583CCDFE9DEE780EF
:1000EE000D89828A83E493A3F608DFF9ECFAA9F06E
:1000FE00EDFB2289828A83ECFAE0A3C8C582C8CCC4
:10010E00C583CCF0A3C8C582C8CCC583CCDFEADEDC
:10011E00E880DB89828A83E493A3F208DFF980CC3E
:10012E0088F0EF60010E4E60C388F0ED2402B40437
:10013E000050B9F582EB2402B4040050AF232345DE
:06014E0082239000AE7355
:10015400BB010689828A83E0225002E722BBFE02A9
:09016400E32289828A83E49322DC
:10016D00BB010CE58229F582E5833AF583E0225047
:10017D0006E92582F8E622BBFE06E92582F8E22291
:0D018D00E58229F582E5833AF583E49322AB
:10019A00BB010689828A83F0225002F722BBFE0144
:0201AA00F3223E
:1001AC00EF8DF0A4A8F0CF8CF0A428CE8DF0A42E67
:0201BC00FE2221
:1001BE00C2D5EC30E709B2D5E4C39DFDE49CFCEE5C
:1001CE0030E715B2D5E4C39FFFE49EFE120586C349
:1001DE00E49DFDE49CFC800312058630D507C3E444
:0601EE009FFFE49EFE22CB
:1001F400BB010A89828A83E0F5F0A3E022500687D6
:10020400F009E71922BBFE07E3F5F009E319228997
:0B021400828A83E493F5F074019322CA
:10021F00BB0110E58229F582E5833AF583E0F5F01D
:10022F00A3E0225009E92582F886F008E622BBFEFA
:10023F000AE92582F8E2F5F008E222E5832AF58340
:08024F00E993F5F0A3E9932205
:10025700BB010A89828A83F0E5F0A3F0225006F7F2
:0F02670009A7F01922BBFE06F3E5F009F31922EF
:10027600F8BB0111E58229F582E5833AF583E8F0BA
:10028600E5F0A3F0225009E92582C8F608A6F02277
:0D029600BBFE09E92582C8F2E5F008F2225E
:1002A300E88FF0A4CC8BF0A42CFCE98EF0A42CFCFA
:1002B3008AF0EDA42CFCEA8EF0A4CDA8F08BF0A478
:1002C3002DCC3825F0FDE98FF0A42CCD35F0FCEBD7
:1002D3008EF0A4FEA9F0EB8FF0A4CFC5F02ECD399C
:0F02E300FEE43CFCEAA42DCE35F0FDE43CFC2209
:1002F20075F008758200EF2FFFEE33FECD33CDCCC3
:1003020033CCC58233C5829BED9AEC99E582984045
:100312000CF582EE9BFEED9AFDEC99FC0FD5F0D622
:10032200E4CEFBE4CDFAE4CCF9A88222B800C1B94C
:100332000059BA002DEC8BF084CFCECDFCE5F0CB8A
:10034200F97818EF2FFFEE33FEED33FDEC33FCEBC3
:1003520033FB10D703994004EB99FB0FD8E5E4F97E
:10036200FA227818EF2FFFEE33FEED33FDEC33FC6B
:10037200C933C910D7059BE99A4007EC9BFCE99A5F
:10038200F90FD8E0E4C9FAE4CCFB2275F010EF2FA4
:10039200FFEE33FEED33FDCC33CCC833C810D707A4
:1003A2009BEC9AE899400AED9BFDEC9AFCE899F8DF
:0E03B2000FD5F0DAE4CDFBE4CCFAE4C8F92272
:1014A000C2D5E830E70FB2D5E4C39BFBE49AFAE477
:1014B00099F9E498F8EC30E717B2D51214D6120374
:1014C0002EE4C39BFBE49AFAE499F9E498F88003CC
:1014D00012032E30D50DE4C39FFFE49EFEE49DFD74
:0414E000E49CFC226A
:1003C000EB9FF5F0EA9E42F0E99D42F0E89C45F093
:0103D000220A
:1003D100E8600FECC313FCED13FDEE13FEEF13FF0A
:0303E100D8F1222E
:1003E400E709F608DFFA807BE9D39850F3E92FF99F
:1003F400E82FF819E718F6DFFA8068E709F208DF52
:10040400FA806080E388828C83E709F0A3DFFA80B6
:1004140052E309F608DFFA804AE9D398500EE92F2F
:10042400F9E82FF819E318F2DFFA8037E309F20844
:10043400DFFA802F88828C83E309F0A3DFFA80231C
:1004440089828A83E0A3F608DFFA801789828A8387
:10045400E493A3F208DFF9800A89828A83E0A3F295
:1004640008DFFA0204F680B180F980A580C680DC3A
:1004740080F180738010808380E98087808780D9B1
:1004840080E180BC8073D3E998EA9C5039E92FF568
:1004940082EA3BF583E82FF8EC3BFC0582D5820227
:1004A40015831582E493C8C582C8CCC583CC058264
:1004B400D5820215831582F0C8C582C8CCC583CC09
:1004C400DFD9DED7802E89828A83ECFAE493A3C82D
:1004D400C582C8CCC583CCF0A3C8C582C8CCC583AB
:1004E400CCDFE9DEE7800D89828A83E493A3F608F2
:1004F400DFF9ECFAA9F0EDFB22D3E998EA9C503835
:10050400E92FF582EA3BF583E82FF8EC3BFC058202
:10051400D5820215831582E0C8C582C8CCC583CCB8
:100524000582D5820215831582F0C8C582C8CCC560
:1005340083CCDFDADED880BC89828A83ECFAE0A33C
:10054400C8C582C8CCC583CCF0A3C8C582C8CCC5F5
:1005540083CCDFEADEE8809C809888F08E83EF60AD
:10056400010E4E608DED2402B404005085F582EB3B
:100574002402B4040050E123234582AB8323900476
:020584006A7398
:10058600BC000BBE0029EF8DF084FFADF022E4CC59
:10059600F875F008EF2FFFEE33FEEC33FCEE9DEC22
:1005A600984005FCEE9DFE0FD5F0E9E4CEFD22ED68
:1005B600F8F5F0EE8420D21CFEADF075F008EF2FB2
:1005C600FFED33FD4007985006D5F0F222C398FDA3
:0505D6000FD5F0EA2240
:00000001FF
